:020000023000CC
:10E000000D9472F00D9493F00D9493F00D9493F0A1
:10E010000D9493F00D9493F00D9493F00D9493F070
:10E020000D9493F00D9493F00D9493F00D9493F060
:10E030000D9493F00D9493F00D9493F00D9493F050
:10E040000D9493F00D9493F00D9493F00D9493F040
:10E050000D9493F00D9493F00D9493F00D9493F030
:10E060000D9493F00D9493F00D9493F00D9493F020
:10E070000D9493F00D9493F00D9493F00D9493F010
:10E080000D9493F00D9493F00D9493F00D9493F000
:10E090000D9493F00D9493F00D9493F00D9493F0F0
:10E0A0000D9493F00D9493F00D9493F00D9493F0E0
:10E0B0000D9493F00D9493F00D9493F00D9493F0D0
:10E0C0000D9493F00D9493F00D9493F00D9493F0C0
:10E0D0000D9493F00D9493F00D9493F00D9493F0B0
:10E0E0000D9493F011241FBECFEFD1E2DEBFCDBF60
:10E0F00001E00CBF12E0A0E0B2E0E0EAF8EE03E0DD
:10E100000BBF02C007900D92A030B107D9F70F9452
:10E11000A3F00D944EF401E20EBF0FEF0DBF1124DA
:10E120001FBE0D94A3F00D9400F020E030E040ED10
:10E1300057E005C0FA013197F1F72F5F3F4F2817DD
:10E140003907C0F308952F923F924F925F926F92DA
:10E150007F928F929F92AF92BF92CF92DF92EF9277
:10E16000FF920F931F93DF93CF93CDB7DEB7C852C3
:10E17000D1400FB6F894DEBF0FBECDBF279A2F9ABD
:10E180008091C00082608093C00080E18093C400D1
:10E1900088E18093C1000000EE24FF248701E4E0C1
:10E1A000AE2EB12CCC24DD2424C0C5010197F1F79B
:10E1B0000894E11CF11C011D111D21E2E2162EE460
:10E1C000F20620E0020720E0120718F071E0C72EE7
:10E1D000D12CC801B70128E53BE140E050E00F94A5
:10E1E0002CF4611571058105910519F485B18058EC
:10E1F00085B98091C00087FD03C0C114D104A9F284
:10E20000A6014F5F5F4FC25EDE4F59834883CE51F8
:10E21000D140C25EDE4F68817981CE51D1406130FC
:10E22000710509F0FCC222243324A0E0C05EDE4F59
:10E230001882C052D1408824992454014424552482
:10E240003201ABBEF40187919691C95DDE4F99838F
:10E250008883C752D140DFC2C25EDE4FE881F981B8
:10E26000CE51D140319709F53091C600C25EDE4FE4
:10E2700019821882CE51D14022C04F5F5F4F6F4F3D
:10E280007F4F4130F2E15F07FAE76F07F0E07F0769
:10E2900080F0C95DDE4F28813981C752D1402F5FA0
:10E2A0003F4F19F0EE27FF27099440E050E060E06F
:10E2B00070E08091C00087FFE0CF3091C6009330BE
:10E2C00061F1943028F4913089F0923008F508C05B
:10E2D000953091F1953040F1963009F043C03EC041
:10E2E0003B3109F0B9CF91E0ABE1B6CF313041F02D
:10E2F000C05EDE4F5881C052D140351709F0AAC226
:10E30000A327C05EDE4F3883C052D14092E0A4CF35
:10E31000132F00E0A32793E09FCF832F90E0082BDB
:10E32000192BA32794E098CF3E3009F093C2A3277E
:10E3300095E02224332490CFE1E0F0E0EC0FFD1FC4
:10E34000E20DF31D30830894211C311CA3272016F5
:10E35000310609F081CF810196E07ECF3A1709F0AE
:10E3600079C203C0973009F077CF8981833109F4EE
:10E37000F4C08431C0F4863009F4C2C0873048F458
:10E38000823069F1833009F45BC0813009F0C4C187
:10E3900041C0813109F465C0823108F0ACC08031E0
:10E3A00009F0BAC11CC0883109F474C0893150F435
:10E3B000853109F4D2C0853108F443C1863109F0B2
:10E3C000ABC13FC18A3109F45CC08A3108F482C014
:10E3D0008B3109F44BC08D3109F09EC102C090E031
:10E3E00041C08D81803311F090E00AC08F81882375
:10E3F00011F49EE105C0813011F091E001C098E96F
:10E400001A821B828D818C831D829E831F8247E02E
:10E4100050E086C11A8288E08B8381E48C8386E594
:10E420008D8382E58E8389E48F8383E5888780E509
:10E4300089878FE58A8782E38B874BE050E070C144
:10E440008A81813941F0823941F0803911F48FE0BD
:10E4500005C080E003C082E001C08AE01A828B839D
:10E4600047C091E01A8242E050E05BC18D81882371
:10E4700011F48EE129C0813011F081E025C088E9D6
:10E4800023C01A82E1E0F0E069E060935700E49174
:10E49000EB831CC08B81803589F48C81883039F402
:10E4A00029E0E2E0F0E02093570084910DC029E0DC
:10E4B000E0E0F0E020935700849106C0E3E0F0E054
:10E4C00039E03093570084911A828B831C8244E098
:10E4D00050E026C18D81836C49E0E1E0F0E0082E38
:10E4E00040935700E89507B600FCFDCF1A821B82C7
:10E4F00043E050E015C11A824424552432010EC174
:10E500008A8190E0A0E0B0E0B82EAA249924882463
:10E510008B8190E0A0E0B0E0DC0199278827882A71
:10E52000992AAA2ABB2A8D8190E0A0E0B0E0882A2F
:10E53000992AAA2ABB2A8C8190E0A0E0B0E0BA2FE9
:10E54000A92F982F8827882A992AAA2ABB2A880CBB
:10E55000991CAA1CBB1C1A82E1C09A813B818331A1
:10E5600019F0B501A40169C050E0451650EC5506FC
:10E5700053E0650650E0750690F463E0F2016092A6
:10E580005B0060935700E89507B600FCFDCF40E0C4
:10E5900051E060E070E0440E551E661E771ECE5DB1
:10E5A000DE4F9883C252D140CF5DDE4F1882C152F8
:10E5B000D140032F10E0CF5DDE4F68817981C152D9
:10E5C000D140062B172BB501A401DE011B968C91BF
:10E5D00011962C9111971296CC5DDE4F2883C45270
:10E5E000D140CD5DDE4F1882C352D14090E0CD5D69
:10E5F000DE4FE881F981C352D1408E2B9F2B21E061
:10E600000C01FA0160935B0020935700E8951124F8
:10E610004E5F5F4F6F4F7F4F02501040C1F635E0A5
:10E62000F401A0925B0030935700E89507B600FC18
:10E63000FDCF81E180935700E8951A824A015B0182
:10E640006DC09A81CA5DDE4F9883C652D140CB5DC2
:10E65000DE4F1882C552D1408B81C82EDD24CB5DA0
:10E66000DE4FA881B981C552D140CA2ADB2A1A825D
:10E6700089818431E9F4A60123E0E22EF12CEC0E2D
:10E68000FD1EABBEF40187919691F70180839183C3
:10E6900022E030E0E20EF31E62E070E080E090E005
:10E6A000860E971EA81EB91E4250504051F72EC02C
:10E6B000B501A40193E0E92EF12CEC0EFD1E0894A7
:10E6C000C108D108860120E030E00894C11CD11CAB
:10E6D0000F5F1F4F2F4F3F4F080D191D2A1D3B1D68
:10E6E00041BDBB27A72F962F852F82BD4F5F5F4F60
:10E6F0006F4F7F4FF89A80B5D7018D937D014017FA
:10E7000051076207730761F74A015B01A6014D5F7C
:10E710005F4FF701108204C0F0ECFA8342E050E052
:10E7200090E02BE12093C6008091C00086FFFCCFD3
:10E730008091C00080648093C000C05EDE4F38814D
:10E74000C052D1403093C6008091C00086FFFCCFFC
:10E750008091C00080648093C000652F5093C600F4
:10E760008091C00086FFFCCF8091C00080648093C0
:10E77000C000342F4093C6008091C00086FFFCCFBC
:10E780008091C00080648093C0008EE08093C600BA
:10E790008091C00086FFFCCF8091C0008064809390
:10E7A000C000A5E1C05EDE4F7881C052D140A727EE
:10E7B000A327A627FE01319610C030813093C600F2
:10E7C0008091C00086FFFCCF31968091C0008064AC
:10E7D0008093C000A327415050404115510569F76F
:10E7E000A093C6008091C00086FFFCCF8091C0003E
:10E7F00080648093C00085B1805885B9992379F4ED
:10E80000C05EDE4F8881C052D1408F5FC05EDE4F58
:10E810008883C052D14090E000E010E01DCD2798E1
:10E820002F9880E090E020ED37E0F9013197F1F783
:10E83000019684369105C9F700008091C0008D7F54
:10E840008093C00081E180935700E895EE27FF2771
:10E850000994FFCF90E000CDA1E21A2EAA1BBB1BAA
:10E86000FD010DC0AA1FBB1FEE1FFF1FA217B3079C
:10E87000E407F50720F0A21BB30BE40BF50B661FB2
:10E88000771F881F991F1A9469F760957095809576
:10E8900090959B01AC01BD01CF010895F894FFCF85
:040000033000E000E9
:00000001FF
